:1000000000180020C1000000F1250000BD250000FF
:10001000BD250000BD250000BD250000BD25000058
:10002000BD250000BD250000BD250000F125000014
:10003000F1250000BD250000F1250000AD250000E0
:10004000F1250000F1250000F1250000F125000058
:10005000F1250000F1250000F1250000F125000048
:10006000F1250000F1250000F1250000F125000038
:10007000312C0000D130000069360000F12500006D
:10008000F1250000F1250000F1250000F125000018
:10009000F1250000F1250000893B0000F12500005A
:1000A000C9130000F1250000F1250000F125000032
:1000B000F1250000F1250000F1250000F1250000E8
:1000C00038B502F099FA454A454B1A60454A464B05
:1000D0001A60464A464B1A60464B0822197811426C
:1000E00002D019780A431A70434B2A221A7000234F
:1000F000424A43499A188A4204D24249C9580433B1
:100100001160F5E7404B41491A1F181D00238A4230
:1001100002D21360031CF6E73D493E4A5958101CB1
:1001200099500433C02BF7D100239A083A49920022
:10013000521803211940C9001568FF248C40A543BB
:100140002C1C80258D40291C214301331160202B5C
:10015000EBD1324B8A221860314B1A70314B24227A
:100160005A70A0221A709A799107FCD59A79D5060F
:10017000FCD498790C212B4A01400829F9D103219C
:100180001171402151719A799106FCD59A795506E1
:10019000FCD52549254A1160224A20211170997900
:1001A0000C220A400C2AFAD1214A224B1A60224A18
:1001B000224B1A60224B00221A60224B07221A603F
:1001C000214A224B1A6062B600F0D6FF04F088FB89
:1001D00002F018FA02F090F9FEE7C046300004F091
:1001E00034800440823F0000388004400100000F4A
:1001F0003C80044002D0074000E00740700200202D
:1002000060040020D855000064040020D8080020B5
:100210000000000000F9FF1F00E400E008ED00E02E
:100220000050064000400640000001104480044099
:10023000C0000505048004407FBB000014E000E01E
:1002400018E000E010E000E00000202020ED00E0D9
:10025000FFFFFFFFFFFFFFFFFFFFFFFFFFFFFFFFAE
:10026000FFFFFFFFFFFFFFFFFFFFFFFFFFFFFFFF9E
:10027000FFFFFFFFFFFFFFFFFFFFFFFFFFFFFFFF8E
:10028000FFFFFFFFFFFFFFFFFFFFFFFFFFFFFFFF7E
:10029000FFFFFFFFFFFFFFFFFFFFFFFFFFFFFFFF6E
:1002A000FFFFFFFFFFFFFFFFFFFFFFFFFFFFFFFF5E
:1002B000FFFFFFFFFFFFFFFFFFFFFFFFFFFFFFFF4E
:1002C000FFFFFFFFFFFFFFFFFFFFFFFFFFFFFFFF3E
:1002D000FFFFFFFFFFFFFFFFFFFFFFFFFFFFFFFF2E
:1002E000FFFFFFFFFFFFFFFFFFFFFFFFFFFFFFFF1E
:1002F000FFFFFFFFFFFFFFFFFFFFFFFFFFFFFFFF0E
:10030000FFFFFFFFFFFFFFFFFFFFFFFFFFFFFFFFFD
:10031000FFFFFFFFFFFFFFFFFFFFFFFFFFFFFFFFED
:10032000FFFFFFFFFFFFFFFFFFFFFFFFFFFFFFFFDD
:10033000FFFFFFFFFFFFFFFFFFFFFFFFFFFFFFFFCD
:10034000FFFFFFFFFFFFFFFFFFFFFFFFFFFFFFFFBD
:10035000FFFFFFFFFFFFFFFFFFFFFFFFFFFFFFFFAD
:10036000FFFFFFFFFFFFFFFFFFFFFFFFFFFFFFFF9D
:10037000FFFFFFFFFFFFFFFFFFFFFFFFFFFFFFFF8D
:10038000FFFFFFFFFFFFFFFFFFFFFFFFFFFFFFFF7D
:10039000FFFFFFFFFFFFFFFFFFFFFFFFFFFFFFFF6D
:1003A000FFFFFFFFFFFFFFFFFFFFFFFFFFFFFFFF5D
:1003B000FFFFFFFFFFFFFFFFFFFFFFFFFFFFFFFF4D
:1003C000FFFFFFFFFFFFFFFFFFFFFFFFFFFFFFFF3D
:1003D000FFFFFFFFFFFFFFFFFFFFFFFFFFFFFFFF2D
:1003E000FFFFFFFFFFFFFFFFFFFFFFFFFFFFFFFF1D
:1003F000FFFFFFFFFFFFFFFFFFFFFFFFFFFFFFFF0D
:10040000FFFFFFFFFFFFFFFFFFFFFFFFDEF9FFFF23
:1004100010B5064C2378002B07D1054B002B02D0DA
:10042000044800E000BF0123237010BD60040020D9
:1004300000000000D855000008B5084B002B03D081
:100440000748084900E000BF07480368002B03D0B5
:10045000064B002B00D0984708BDC04600000000A6
:10046000D855000064040020600400200000000053
:1004700010B5041C00F042FE2368C01A10BDFFFF37
:1004800010B50948FFF7F4FF084C20600E2000F07B
:10049000DFFDA36841424141C9B201330C206160D4
:1004A000A36000F0B5FD10BD100500209C040020E5
:1004B00008B5011C014802F013F808BDEC04002047
:1004C00008B5011C014802F004F808BDEC04002046
:1004D00000B58DB0021C084904A804F015FB04A95E
:1004E000684601F077FF6846FFF7EAFF684601F0CB
:1004F0002DFF0DB000BDC0469451000000B58DB079
:10050000021C084904A804F0FFFA04A9684601F097
:1005100061FF6846FFF7D4FF684601F017FF0DB092
:1005200000BDC0469851000030B5134B85B01D7812
:10053000124C002D0AD02068A16801F033FB01F0B5
:1005400063FB201CF02101F07FFF12E00C48A26841
:10055000036821685B68984701F086FD291C68469E
:1005600001F038FF201C694601F066FF684601F083
:10057000EDFE05B030BDC0460C050020EC040020A7
:100580009806002008B5054B0A201B78002B00D0E8
:10059000F720FFF78DFFFFF7C7FF08BD0C05002010
:1005A00010B5141CCAB01A0CD2B2031C00910194ED
:1005B0000AA8084904F0A8FA0AA906A801F00AFF47
:1005C00006A8FFF77DFF06A801F0C0FEFFF7DAFFDF
:1005D0004AB010BD9C510000031C413B192B01D8AF
:1005E000203004E0031C613B192B01D82038C0B235
:1005F000704708B5FFF7F0FFFFF75AFFFFF7C2FF9C
:1006000008BDFFFF10B5054C0021201C2C2204F072
:10061000B9F901235B42636010BDC046BC040020F1
:1006200010B572B6FFF7EEFF00240D4B0021E05825
:100630001022043404F0A6F9142CF6D1094B4C22F4
:100640009A73094B53229A73084B47229A73084BAB
:1006500041229A73074B4D229A7362B610BDC04671
:10066000740200209C04002014050020FC040020DB
:10067000AC0400207C04002010B50B20012100F008
:10068000F9FC0C20012100F0F5FC0D20012100F007
:10069000F1FC1420002100F0EDFC0F20002100F0FF
:1006A000E9FC1020002100F0E5FC0E20022100F002
:1006B000E1FC0E200C49042200F06CFC0B4B0022E4
:1006C0001A700124FFF7ACFF094B211C0D201C7090
:1006D00000F09EFC211C0B2000F09AFC0C20211C39
:1006E00000F096FC10BDC046810400000C050020FF
:1006F000E804002030B50B2085B0012100F088FC13
:10070000FA24A400142000F097FB051C1248FFF700
:10071000AFFEFFF7DDFE2020FFF7CAFE28B2FFF78D
:10072000D7FEFFF72FFFE1235B01013BFDD1013C29
:10073000002CE7D1211C0B2000F06AFC0749684619
:1007400001F048FE6846FFF7BBFE684601F0FEFD7B
:10075000FFF718FF05B030BD10050020AB510000B9
:1007600030B50B2085B0012100F052FCFA242401A1
:10077000102000F061FB051C1248FFF779FEFFF71F
:10078000A7FE2020FFF794FE281CFFF7A1FEFFF72D
:10079000F9FEE1235B01013BFDD1013C002CE7D1D7
:1007A000211C0B2000F034FC0749684601F012FEC2
:1007B0006846FFF785FE684601F0C8FDFFF7E2FED8
:1007C00005B030BD10050020AB5100007FB5041E00
:1007D0005A2C16D172B600F091FCB64B1860FFF798
:1007E00011FFB54B01221A7062B60025B34B291CCC
:1007F0000B201D7000F00CFC0C20291C00F008FCE4
:1008000018E054280FD1AE49684601F0E3FD684670
:10081000FFF756FE684601F099FDA648FFF728FE4F
:10082000FFF76CFE42E1502804D0442806D10A208C
:1008300000F088FC201CFFF7DCFE39E1031C313B93
:10084000082B0AD89B48FFF713FE2F3C9A4B012236
:10085000A4005242E0505A602AE1522811D1964A2F
:1008600000245368591C5160082902DCD91C8900F6
:100870008C58981CFFF72CFE3A20FFF719FE201C1D
:1008800004E1492819D18C4B012252425A600024BC
:100890001D1C8C4B013BFDD18648FFF7E9FDA300F1
:1008A000EB189860201C3130C0B20134FFF700FE15
:1008B000FFF768FE092CECD1FAE0462802D1FFF7D9
:1008C000AFFEB7E7562811D1FFF786FEFFF7F0FD20
:1008D0002020FFF7EDFD7C49684601F07BFD68466E
:1008E000FFF7EEFD684601F031FDDFE047280BD150
:1008F000764C2068FFF7ECFDFFF744FE00232360F1
:10090000A36001232373D3E0412801D1704B1DE084
:10091000422812D16748FFF7ABFD6E490022051C43
:10092000172001F051FC201CFFF756FEFFF7C0FD19
:100930002020FFF7BDFD281CA8E0532803D1172075
:1009400001F0D6FC76E74D2807D1634B00221A60F0
:100950009A6001221A735A736CE74E2820D1554EC3
:100960005E4A316868468B180093FFF781FD051CCD
:10097000201CFFF731FEFFF79BFD2020FFF798FDBD
:10098000281CFFF7BBFDFFF7FDFD301CFFF770FDD6
:10099000A842FAD3524801F0BBF801F035F987E0DC
:1009A00043280ED1142000F047FA4E4C0123191CA5
:1009B000221C6E2800DC00236360517311734320F6
:1009C00039E7632804D1474B00225A731A7331E781
:1009D000452801D1434C11E04C2805D1424B01225E
:1009E0005A7300229A6025E76C2804D13E4B0022FE
:1009F0005A736C201FE74A2809D13B4CE3682068F2
:100A00006168A268FFF7CCFD0023A36050E0552881
:100A100004D1FFF7EEFDFFF76DFE49E04F2804D14A
:100A2000FFF7E7FDFFF79CFE42E0512831D1FFF7C9
:100A3000D3FDFFF73DFD2D49684601F0CBFC68462C
:100A4000FFF73EFD684601F081FC0F2000F0F4F94D
:100A5000FFF73EFD2649684601F0BCFC6846FFF7FB
:100A60002FFD684601F072FC142000F0E5F9FFF755
:100A70002FFD2049684601F0ADFC6846FFF720FDD8
:100A8000684601F063FC0E2000F0D6F9FFF720FD68
:100A90000CE01949684601F09DFC6846FFF710FD1F
:100AA000684601F053FC201CFFF702FDFFF76AFDCA
:100AB0007FBDC04610050020BC040020E8040020D3
:100AC000AF510000102E0000B2510000FC040020C5
:100AD000AC040020881300007C040020F0D8FFFF45
:100AE00009903C63140500209C040020B4510000D0
:100AF000B8510000C4510000CF510000F0B5624C65
:100B000087B021780D2000F083FA604D2B7B002BFD
:100B100013D00F2000F090F9E1239B0098420CDDE8
:100B20005B48FFF7A5FCAB6801220133AB600023F3
:100B30002B732378286053402370564D2B7B002B5A
:100B400011D0162000F078F914280CDD5048FFF77A
:100B50008FFCAB6801220133AB6000232B73237839
:100B6000286053402370012001F068F8061C701EB5
:100B70008641F6B20196002E07D0474D2B7B002B05
:100B800003D0464B1F78002F6ED0454D2B7B002B9A
:100B900019D0142000F050F96968002902D16E289C
:100BA00002DC10E059280EDC3948FFF761FCAB6825
:100BB00001220133AB6023786E6853402370734287
:100BC000734128606B60002472B6364B0021E358F5
:100BD0005A7B8A420BD09F688F4208DD324A1D1C27
:100BE000101CC4CDC4C02D6805609960012162B697
:100BF000002906D02C4B186859689A68DB68FFF703
:100C0000CFFC0434142CDFD1019E002E22D0234BC4
:100C10001B78042B18D1254B02A8197801394B42B7
:100C20005941234BC9B21970002903D0F02101F0BA
:100C300015FC01E001F0CEFB02A91E4801F0FCFB0F
:100C400002A801F083FB05E0052B03D1174B1878B0
:100C5000FFF7BCFD01F066F9002812D001F01AF987
:100C6000C0B2FFF7B3FD0CE00948FFF701FCAB6829
:100C700001220133AB602378286053402F73237027
:100C800083E707B0F0BDC046E8040020FC04002064
:100C900010050020AC0400207C0400208608002001
:100CA00014050020740200208C0400208808002015
:100CB0000C050020EC04002010B500F01FFA064BD4
:100CC000064C18600021201C01F084FB201C044904
:100CD000044A03F0EDFD10BD10050020EC040020D7
:100CE0004D23000070020020F0B51E4B1A688023CF
:100CF0001A40FAD172B61C4B1978002930D01B4922
:100D00000C681B490F681B493C190E681A49A41945
:100D10000D681A496419086819492418096819489E
:100D20006418A4B2184964080C43A4B20460174CB8
:100D3000174800682568174CAC462768164C604475
:100D40002668164CC0192568154C8019246840196E
:100D5000001980B240080143124889B201601A703C
:100D600062B6F0BD24B003402505002038B0034032
:100D70003CB0034040B0034044B0034048B003409F
:100D80004CB003402CB003400080FFFF5CB0034038
:100D900058B0034060B0034064B0034068B0034003
:100DA0006CB0034030B003401B4B1C4A19781C4BFD
:100DB000082901D1002102E00A2903D1382111605C
:100DC000132206E00C2901D1342100E03C211160FE
:100DD00012221A60134B1A78134B002A01D00022FA
:100DE00000E001221A60114B1A78114B012A01D838
:100DF00080220CE0042A01D8842208E0082A01D8C5
:100E0000852204E0102A01D8862200E087221A6099
:100E1000084B01221A7070478802002008B0034076
:100E20000CB003402705002020B0034089020020B9
:100E300024B0034025050020031C70B50020272B9B
:100E400032D81A4AD45CFF2C2ED0194B1B7883421F
:100E500001D0FFF749FF72B6164B1022610605D587
:100E60001968914319603F231C4002E019680A4346
:100E70001A60114B114D01221C602A7062B61E1CB3
:100E800072B633681A0608D50D4B186800232B700C
:100E900062B60C4B1B78184106E02B78002BDBD098
:100EA00062B601F05FFBEBE770BDC046E1510000A8
:100EB000250500200CB0034000B0034026050020AB
:100EC00010B00340240500207047FFFF38B5074BE2
:100ED0001C681C60064BDA681D1CA30700D59047F0
:100EE0002B69620700D5984738BDC046A0900440E2
:100EF0008C02002038B5244B244C1D681D60636AA9
:100F00002A0700D59847A36AEA0600D59847E36AFE
:100F10006A0600D59847236B2A0600D59847636B6D
:100F2000AA0600D59847E36BEA0700D59847A36D5A
:100F3000AA0700D59847E36D6A0700D59847144B78
:100F40001D681D60A368EA0700D5984763692A06F3
:100F500000D59847A369EA0600D59847E3696A0770
:100F600000D59847236A2A0700D59847A36BAA079C
:100F700000D59847236DAA0600D59847636D6A0689
:100F800000D5984738BDC046A0B004408C02002070
:100F9000A0C0044070B5041E1A2C2CD8042A2AD8EC
:100FA000101C02F0BDFE0709050B03000B2306E031
:100FB0000A2304E0082302E00C2300E009230C22AA
:100FC00062430D480D4E82180D485268051CB83515
:100FD0002E600C4DBC30056072B60B481568A4003D
:100FE00028400A4D106061518021490408431B04C8
:100FF0001843106062B670BD0C520000CD0E0000A8
:1010000000F9FF1FF50E0000FFFFF0FF8C0200202B
:1010100010B51A2818D80C2358430C4A83581018B6
:101020001C7D027A224205D0002901D01A710BE002
:101030001A7209E043681A68002902D003210A43A2
:1010400001E002218A431A6010BDC0460C52000024
:1010500000231A280AD80C235843054A815810182F
:10106000027A0B7C13405A1E9341DBB2181C704766
:101070000C520000F0B51A283DD80C273D1C454302
:101080001D4A54196368161C012901D0042912D184
:10109000784332583018147D007A20431075A2220C
:1010A00052001A602022042901D1196814E019683D
:1010B00091430A1C1EE0AA58247A107DA0431075A3
:1010C000002902D08A1E012A12D8802252001A60FA
:1010D000022903D11A6803210A430BE003290AD12C
:1010E0001A6802210A431A601A6801218A4301E042
:1010F0000422FF321A60F0BD0C52000072B60C4B95
:101100000C491A680C4B1B68096862B6480104D583
:1011100032219142894149425B18FA2080004343C1
:101120000648821A06484243920D98187047C046F6
:1011300018E000E004ED00E0280500207FBB00007F
:101140005555010038B5041CFFF7D8FF051C002CCD
:101150000FD0FFF7D3FF074B401B984206D9013C45
:10116000002C06D0FA239B00ED18F2E701F0FAF903
:10117000EFE738BDE70300001D4B8022D20510B514
:101180001A60802212061A601A4B002018601A4951
:101190001A4B1B4A1960282313601A4A1A4C136011
:1011A0001A4A13601A4A13601A4A13601A4A1360E3
:1011B00009222260194C2060194C2160194C2360CF
:1011C000194C2360194C2260194C206019480160A9
:1011D00019490B6019490B60194B1A60FFF7E4FDC0
:1011E000C8204000FFF7AEFF00F0D8FB10BDC0469E
:1011F00000E100E004800340FFBF000008800340DE
:101200000C80034014800340008003401C80034096
:10121000248003402C80034034800340049003402A
:10122000089003400C90034014900340009003404A
:1012300004A0034008A003400CA0034014A00340F6
:1012400000A00340F0B50B4F02223B780A4E1A4330
:10125000D2000A4DB418606028788824002800D095
:10126000C82409040C43B450012250405340287054
:101270003B70F0BDA005002000F8FF1F20060020F5
:10128000431E10B5042B0FD872B6084A990088582F
:10129000002807D044685B008C50054A01889C5A9E
:1012A000611A995262B600E0002010BD8C05002042
:1012B0007C080020431E0020042B09D872B6054A82
:1012C0009B009B58002B02D001305B68FAE762B6A6
:1012D0007047C046E405002038B572B60123164AAF
:1012E0009A18013A127811071CD5144A5C01A558C6
:1012F0009900002D05D1131908305860104BA350E8
:101300000AE001242143C9008C58002C0AD153184B
:10131000083058600B4B8B500B4B1A78013A1A70FF
:1013200062B608E00133062BD9D162B6064B002223
:101330001A7000F0A7FB38BD7853000000F8FF1FBB
:1013400088004000C800400016060020421E10B56C
:10135000042A30D8022380001843174BC0001B1802
:1013600072B6164CA05C032809D802F0D9FC14020E
:1013700016050833022011E0083304200EE010485F
:10138000920014580F4B002C01D1115001E09858D5
:10139000416099500EE0032000E00520A0540A1C93
:1013A00008325A608822180700D5C8220988090423
:1013B0000A431A6062B610BD00F8FF1F4405002002
:1013C000E4050020F8050020F7B5B6490C780E1C9E
:1013D000E4B262071FD5B44B1B78002B18D0B34A78
:1013E0001378DBB2002B05D0013BDBB21370002B6E
:1013F00000D100BEAE4A1378DBB2002B06D0013B11
:10140000DBB21370002B01D100F05CFE00F0FCFB9E
:10141000A44D04232B700825221C2A4000D154E23D
:10142000A44BA54C1B78DBB21E099A08002E00D0F5
:10143000DDE1D50065192F686A68B806000F01382C
:101440000C2800D9D0E102F075FC93019301CF0183
:10145000CF01CF01CF01CF01CF01AC01CF01CF012F
:10146000CF010D0095491368954F52689548296042
:10147000954D964900263B607A609BB201222E6012
:101480002661A66102708B4218D8D021C9008B4218
:1014900000D3E5E0812191408B4200D1C2E006D823
:1014A000802B00D1A9E0822B00D1ABE0F5E0884A87
:1014B000934200D1C5E0A022D20017E085498B42BB
:1014C00000D152E10DD8882109018B4200D18EE074
:1014D00090221201934200D0DFE0BA78724B1A706A
:1014E00009E07D4A934200D1CFE07C4A0026934236
:1014F00000D115E1D1E0A319196A090603D5586A8C
:10150000083800F0BFFA0836A02EF4D100252E1CB2
:10151000734AA858002805D04368019300F0B2FA36
:101520000198F7E76E496F4B6F4A4851E850A85849
:10153000002805D04368019300F0A4FA0198F7E76A
:101540006A4B6B4AE8507300D0526749694B485167
:10155000F05C0238032807D802F0E2FB0204020420
:10156000002200E001229A5501360435052ECFD124
:10157000614A002313700125161C604BEA18604B6A
:101580009200EB18013B1B781370190720D500F06F
:101590005BFA6B01002805D0E21808305060594A08
:1015A000E25003E0E05033780133337000F04CFA3E
:1015B0000122AB001343DB00002805D0E2180830FD
:1015C00050603E4AE25003E0E0503378013333701C
:1015D000AB0002221A43D2000021A1500322134380
:1015E00093400135E150062DC7D10E1C98E02E4BDB
:1015F000454C1B78161C237093E0434C2670667094
:1016000002268EE0BB88052B47D83F4C3F4D9B0000
:10161000267066705B191B780226334200D180E089
:1016200022707EE0BA887F231340052B35DC7E884C
:10163000002E32D135499B005B181A7802218A436B
:1016400029E0BA887F231340052B26DC7E88002EF4
:1016500023D12E4A9B009B181A7802210A431AE0D4
:101660007A88B9882A4B5C68002C16D0188890427A
:1016700009D15888884206D1120A032A01D1267856
:101680004FE01E894DE00C33EDE7224B1A68224BE8
:101690001A60BA78214B1A7042E01C4B0F221A7064
:1016A00063E0C046802007401F060020A1050020FF
:1016B0005C0600209020074000F8FF1FC800400093
:1016C0000C060020200600202C05002081060000CA
:1016D000020300002120000021220000212300003D
:1016E0008C05002030050020E4050020F8050020CE
:1016F0007C080020440500201606002030C8011098
:10170000785300008800400017060020C0200740E2
:101710008053000028050020D00800206C0600201F
:10172000341CFB889E4200D91E1C371E402F00D956
:101730004027201C391CFFF785FDE419F61B03D157
:10174000351C402F04D010E04025B54200D9351C8F
:10175000201C291CFFF776FD6419761B01D1402D52
:1017600003D1754D754B2C601E800122744B3AE0FD
:10177000744B1988744B994210D10023D05C734983
:10178000C8540133072BF9D10B68862B02D1704B5B
:101790000F221A700020011CFFF754FD6D4B2B60C7
:1017A00022E0654F3D68002D13D064490E88341E39
:1017B000402C00D94024281C211CFFF743FD361B78
:1017C0005E4AB6B21680002E01D1402C00D12E19EF
:1017D0003E605C4BA0221988D200914204D10022C5
:1017E0005A709A785C4B1A700122554B61E0D20016
:1017F000A4186068013E0838F6B22B4036D000F0DD
:1018000041F95649B0004258554B002A1BD0556843
:101810004550111C985D0831616003280BD802F017
:101820007FFA02040608032104E0022102E00521F8
:1018300000E0042199558823270700D5C823128882
:10184000120413433CE0985D032808D802F068FABC
:1018500039390204002200E001229A5531E02C407F
:10186000624262410324A41A9C552AE062880280E5
:10187000002A20D03B4D43804360B3005F593A4972
:10188000002F01D1585101E0CD586860C850374B46
:101890007600F15A5218F25200F0D6F8002804D01F
:1018A0000830606021070AD507E0314B20601A78C4
:1018B00001321A7005E02C4201D0264B00E02D4B7E
:1018C00023602D4A082313707FE5012004421ED0B7
:1018D0001B4902230B70294B264C1A70284B294DAB
:1018E0001C609C60284C1A61DC609A615D60274B2B
:1018F0000D241C70264CFF232370174C337022706C
:10190000244A1370244B9F221A70087013E063B2AC
:10191000002B04DA1D4B0D221A7080233370022332
:101920001C4204D01A4A1178C9B2117033701023C6
:101930001C4200D03370F7BD2C0500201406002097
:10194000942007400C06002021200000C808002039
:10195000A1050020C800400098200740E4050020B1
:10196000440500208C050020300500207C08002064
:10197000160600208800400080200740A0050020B7
:1019800000F8FF1F4C050020A4050020C0200740E0
:10199000882007408C2007408420074010B501F0C4
:1019A000D9FE00221A4B0021D1509818083241600C
:1019B000A82AF7D1174A80201468C002204310607B
:1019C000180A154AC0B21070180C144AC0B2107030
:1019D000134A1B0E1370134AFF231370124A134845
:1019E0001370134A137001220270124801701249D9
:1019F0000A70124A116899430B1C70210B43136043
:101A00000F4B802252041A600E4B10221A7010BD28
:101A100000F8FF1F348004409C200740B02007409E
:101A2000B4200740802007408820074094200740CA
:101A300010200740002107408420074018E400E000
:101A400000E100E00821074038B572B60B4C25686C
:101A5000281C02F003FA1D2802D962B600200CE00F
:101A600080231B06C3409D43256062B6482358432C
:101A7000034B181800230360436038BDF8020020B0
:101A800000FAFF1F10B5041C0E484821201A02F06E
:101A90005BF91D2815D80C4B1B78002B07D00B4B7E
:101AA0001B78002B03D0201CFFF716FC09E072B650
:101AB0008022074B1206C240101C1A68104318609F
:101AC00062B610BD00FAFF1F160600201F06002098
:101AD000F802002038B50B4C051C21783C2908D1B0
:101AE000094B1B68002B04D00848002298470023AC
:101AF000237023783B2B03D85A1C2270034AD554F9
:101B000038BDC046870800204C0600208B08002006
:101B1000F8B51F4D1F4C01232B702368061C002BAA
:101B20001DD11D4F1D4B1B78002B2FD00420FFF71C
:101B3000C1FB052804D9013F194B002F06D108E04D
:101B4000FFF782FF20600028F5D008E01A78002A0D
:101B500002D001221A7019E000F004FDE2E7104BF8
:101B6000002221681A704A88531C92008A189660D5
:101B70000F2B01D84B8007E040230B800420FFF798
:101B8000E5FBFFF761FF206000232B70F8BDC04626
:101B90003C06002044060020E14200001F06002011
:101BA0004806002038B5041C0D1C032D0ED92078E2
:101BB000637800021B04184304231843A378033DF1
:101BC0001B061843FFF7A4FF0334EEE7032D09D1EA
:101BD0002078637800021B04184307231843A37876
:101BE0001B060DE0022D06D12078637800021B044D
:101BF0001843062304E0012D05D1207805230002B7
:101C00001843FFF785FF38BD10B50A4B1B78002B32
:101C10000ED1094C216800290AD04B88002B07D02F
:101C20009B000B800420FFF791FBFFF70DFF206066
:101C300010BDC0463C06002044060020F8B5834C89
:101C4000071C2368251C002B12D1814B1B78002B0D
:101C500000D1E2E00520FFF713FB2060002800D14F
:101C6000DBE00688002E03D1FFF70CFF2660D4E0EE
:101C7000286843889A08920082189468028804337E
:101C8000934201D2438005E0FFF7FCFE0520FFF7F9
:101C9000F7FA28600F23251C1D40200A061C2A1C69
:101CA0001E40083A0136062A00D980E0002F02D0F3
:101CB000B74200D0B1E0220B1340082D0AD1082B07
:101CC00000D0AAE0634B00221A70634B1B6893425A
:101CD00032D163E0092D1AD1092B00D09DE0220EEC
:101CE0005C4B210C002A09D0012018705B4B1B684B
:101CF000002B53D0F0B2C9B2D2B206E01A70564BE4
:101D00001B68002B4AD0F0B2C9B2984746E00A2DB2
:101D100007D10A2B00D080E04E4B02221A70504BA4
:101D200007E00B2D0DD10B2B77D14A4B03221A70F4
:101D30004C4B1B68002B31D0210CF0B2C9B2220EE3
:101D4000E3E70C2D06D10C2B67D1424B04221A700D
:101D5000454B07E00D2D0DD10D2B5ED13D4B0522DE
:101D60001A70424B1B68002B18D0210CF0B2C9B27C
:101D7000984713E00E2D50D10E2B4ED1354B062235
:101D80001A703B4B1B68002B08D0FE21620C8901A6
:101D900011406202520EF0B211439847354B220CAB
:101DA0001E70354B240E1A70344B1C704CE0042D01
:101DB00008D1C0B2FFF78EFE200CC0B2FFF78AFE3A
:101DC000200E28E06B1F022B1ED8C0B2FFF782FE48
:101DD000052D08D0200CC0B2FFF77CFE072D02D1E4
:101DE000200EFFF777FE264B234A19781170002248
:101DF0001A70184B07221A70224B1B68002B23D035
:101E00002148012298471FE00F2D12D11C4B1B784F
:101E1000002B04D0C0B2FFF75DFE002015E00D4B93
:101E200008221A70194B1B68002BB7D0C0B2984714
:101E3000B4E7022DF1D1074B09221A70144B1B682D
:101E4000002B01D0200C98470120F8BD500600203F
:101E50001F060020860800202806002058060020C3
:101E600034060020540600202C06002038060020EE
:101E7000300600208A0800208808002089080020F9
:101E8000870800204C0600208B0800204006002018
:101E90002406002038B5114C2368002B0CD0206894
:101EA0004288531C8218157A0288934212D3FFF796
:101EB000E9FD002323600EE0094B1B78002B02D1C3
:101EC0000120404208E00220FFF7DAF920600028F4
:101ED000E5D1F5E74380281C38BDC04668060020E0
:101EE0001F06002010B50D4C2368002B03D023687B
:101EF000002B0ED103E00A4B1B78002B02D10120EE
:101F0000404209E00220FFF7BBF920600028EED133
:101F1000F5E75A889B18187A10BDC046680600205D
:101F20001F060020054B5888054B1B68002B03D06B
:101F30001A885B88D31AC0187047C0467C080020F6
:101F40006806002010B50A4B1B78002B0FD0094CF7
:101F50002068002803D0FFF795FD002323600220AE
:101F6000FFF78EF9002802D0FFF78CFDF7E710BDD0
:101F70001F06002068060020F7B5304D0123071C1E
:101F80000C1C2B70002C56D02D4E3068002827D109
:101F90002C4A01922C4B1B78DBB2002B03D12B7007
:101FA0000120404249E00320FFF784F9072808D8C0
:101FB00001232B70FFF748FD214B186000280FD13B
:101FC00028700198214B01380190002802D01A781E
:101FD000002A02D001221A70E2E700F0C3FAD9E722
:101FE0001A4B002231681A704B884020C01A0094A6
:101FF000844200D90090181C009A08309B180818D9
:102000004B800190A41A00230098834204D0F85C0E
:10201000019AD0540133F7E7FF184B883F2B06D9BC
:1020200040230B800320FFF791F900233360084B16
:1020300005221A70A6E72C70201CFEBD5D0600204C
:1020400060060020097500001F06002064060020BD
:102050005C06002007B56B46D8710733181C0121B8
:10206000FFF78AFF0EBDFFFFF8B5124B1B78002B60
:102070001ED0114F114B3C6801261E70104D002CD4
:1020800009D000262E70638803202380211CFFF7CF
:102090005DF93E6009E0FFF7D7FC011E04D0032084
:1020A0002C70FFF753F900E02E70044A00231370E0
:1020B000F8BDC0461F060020600600205D06002017
:1020C0005C06002038B50E4B1D78EDB2002D15D101
:1020D0000C4C2168002906D04B8803200B80FFF7A9
:1020E00035F925600AE0FFF7AFFC011E03D003209D
:1020F000FFF72CF902E0044B01221A7038BDC046EC
:102100005D060020600600205C06002010B5041C5F
:1021100001F0FCFD201C10BD214B70B518681E1C81
:102120002049214A002809D0127809680A71421E04
:10213000511D01D1032252421A6030E00B6812781F
:102140001A4D1A702B68002B23D0194B00211C68E4
:10215000201C01F065FE002816D1201C154901F055
:1021600069FE002810D11449201C02F091F8FC21CE
:10217000890502F0B7F901F08FFE021E272A03D964
:102180000E480F4901F0AAFD2B68336000232B6035
:1021900005E00A4801F0BAFD0A4BFF221A7070BD33
:1021A00090060020840600208C060020880600206F
:1021B00094060020ABAA2A4D0000C0417006002002
:1021C00019210000FC020020F8B5051C0C1C1A287F
:1021D00074D8002A08D0101C4843FA21890001F065
:1021E000B3FD4600013601E003267642201C02F0D2
:1021F0000FFB011C324801F067FE0C236B43314A90
:10220000041CD3185F6872B62F4B19788D4215D114
:102210002E4D296801F0F4FD2D4B002806D01868DA
:1022200001220240013A96191E6046E0294A1968C7
:10223000166001220A402C601A603EE0264B1A29E3
:1022400003D826491868097801701F490D700C21C0
:102250004D4351595519081C083018601F4A287AF7
:102260001070087272B61B681278197B0A431A73D1
:1022700062B6A2235B003B60154B201C1E60134B13
:1022800000211C6001F0CCFD002816D1201C14494F
:1022900001F0D0FD002810D11249201C01F0F8FFF8
:1022A000FC21890502F01EF901F0F6FD021E272A25
:1022B00003D90D480D4901F011FD62B6F8BDC046C5
:1022C0000024F4480C520000FC0200209406002078
:1022D0009006002088060020840600208C0600203E
:1022E000ABAA2A4D0000C041700600201921000051
:1022F00010B51A280FD872B6074C2378834209D13B
:10230000064801F003FD064B064A1B6812781A7056
:10231000FF23237062B610BDFC020020700600206F
:10232000840600208C06002008B5054800230370B1
:1023300004498023044A437302F0BAFA08BDC04638
:10234000700600200D2100007002002010B5041C52
:10235000006802F0EBFA201C10BD38B5041C0D1CFF
:102360000068013102F0B2FB002801D021C4012035
:1023700038BD436810B5041C8B4208D2FFF7EDFF4F
:10238000002805D0A368002B01D12268137001201A
:1023900010BDF8B5041C0F1C151E05D10368002BD9
:1023A00000D01A7000230DE0111CFFF7E2FF061C9D
:1023B0002068002E08D1002802D002F0B7FA26606B
:1023C00000236360A36003E0A560391C02F0BEFB3C
:1023D000201CF8BD38B50023041C0D1C03604360AD
:1023E00083600373994207D0081C02F0B7FB291CD5
:1023F000021C201CFFF7CDFF201C38BD38B5051C82
:1024000000680C1C00280CD06A688B689A4206D3BE
:10241000096802F09BFBA2680023AA600AE002F0B0
:1024200085FA236862682B60A3686A60AB6000234A
:1024300023606360A36038BD10B5041E8C4201D0D8
:10244000FFF7DCFF201C10BD07B5002201AB19709F
:102450005A70191C0122FFF79CFF0EBD10B5002316
:10246000041C0360436083600373FFF7EDFF201CCF
:1024700010BDF7B50368171C0022041C0D1C8668EC
:102480000092994206D39A19914203D2CB1A019332
:1024900001230093002F1AD0BE19201C311CFFF716
:1024A00068FF002813D0009BA0682168002B09D08A
:1024B000019A081889183A1C02F042FA226800238F
:1024C000935503E00818291C02F040FBA660201C6D
:1024D000FEBD08B50B1C9A680968FFF7CAFF08BD66
:1024E00013B5002201AB041C19705A70191C01228B
:1024F000FFF7BFFF201C16BD08B5FEF7BDF8FEF7BD
:10250000FDFA00F02FF8FAE708B5FFF70BFD08BD5C
:1025100008B5FFF7BFFC08BD08B5FFF7E3FC08BD31
:1025200008B5FFF7A1FD08BD08B5FFF70BFD08BD15
:1025300008B5081CFFF78EFD08BD08B5081C111C66
:10254000FFF71AFD08BD7047044B00221A711A7379
:10255000FA21034A890099601A60704798060020A2
:102560005853000010B5104C2378002B1BD10123C9
:102570002370FFF7D7FC002801D0FFF7E4FF00F03D
:10258000E5FA002801D001F0AFF900F02FFD002896
:1025900001D001F049FA00F0F5FF002801D001F068
:1025A000E3FA0023237010BDA8060020024B1A682E
:1025B00001321A607047C0462805002010B50B4C48
:1025C00023685A0301D5FEF7FFFE23685A0501D59B
:1025D00000F02EFB23681A0501D500F079FD236871
:1025E000DA04ECD501F040F8E9E7C0463480044055
:1025F00008B5FFF7E3FFFFFF014B00221A607047A9
:10260000008104407047FFFF024A136818181060E9
:10261000181C704700030020EFF31380002821D11D
:10262000EFF31082002A1FD1EFF30583002B0FD0A8
:10263000101C0F2B0ED91A1C103A92080B490320BC
:1026400092000340521883401068D840C0B201E0A5
:1026500080204000EFF31182002A05D0824203D28D
:10266000101C01E0012040427047C04600E400E039
:10267000F8B5061C0D1C171C0024301C391C01F079
:10268000A7FB092901D8303100E03731C9B22955FB
:10269000301C391C01F058FB061E01D00134ECE758
:1026A0002B1958702B1C5A1BA24206DA1A78295D86
:1026B00019702A550133013CF5E7281CF8BDFFFFCE
:1026C000264B80221968D2000A431A60244A00234C
:1026D0001370244A1370244A1370244A1370244A36
:1026E0001370244B1B78032B09D0152B04D0002B1F
:1026F00008D1214A214B04E01F4A214B01E0214A25
:10270000214B1A60214B1B78042B0BD0052B05D0D5
:10271000012B0BD1D12292001D4B06E0D122920059
:102720001C4B02E091221C4B92001A601B4BC2040E
:10273000D20E1A70C0B2002258709A702C22DA7031
:10274000174BFF22196891430A1C40210A431A6063
:10275000144B802252011A607047C04634800440F6
:1027600035070020B10600203C0700203607002076
:10277000B0060020F20600201303000040A0044031
:1027800018C0044013020000049004400403002019
:1027900044A004401CC004400890044000A006402F
:1027A0000CE400E000E100E010B5174B132299782B
:1027B0009143032202400A43410701D510210A43F5
:1027C0009A700F2210490240042A03D18A794024CA
:1027D00022438A715A7910218A43084200D00A4361
:1027E0005A71997910229143840600D51143064A03
:1027F0009971C10506D5537811782020DBB20143C9
:102800001170537010BDC04600A0064008B5124BB1
:102810001B685A051ED5114B1B78DBB2002B02D06A
:10282000FFF7A0FEF7E70E4A8021490111600D4A2B
:102830000D49D3700422FF320A600C490A600C4A29
:1028400013700C4A13700C4B1B68002B02D00B4A00
:1028500012781A7108BDC04634800440B0060020CA
:1028600080E100E000A0064040A0044044A00440F5
:1028700035070020B1060020AC060020F30600203A
:1028800038B5041C0B4B1D78EDB2002DFAD1201C7D
:102890000121FEF7EFFB291C201CFEF7B9FB0C22DF
:1028A0005443054B054AE1581C191160044B227A28
:1028B0001A7038BDB00600200C5200003807002006
:1028C0003407002030B5002901D080231843224A64
:1028D0001378141C98423ED0204A1268550539D509
:1028E0007F221340042B0FD004D8012B0FD10022DC
:1028F0001B4B0BE0052B04D0182B08D10022194BE1
:1029000004E00022184B01E0184B00221A60442317
:10291000002900D060237F220240042A15D006D867
:10292000012A17D1C022920013430D4A11E0052A53
:1029300006D0182A0ED18022D2001343094A08E09B
:10294000C02292001343084A03E0802292001343FE
:10295000064A1360207030BD040300203480044018
:1029600044A0044050D004401CC0044008900440DF
:1029700010B51A4A137898422ED0194909684C05A7
:1029800029D5032B0FD004D8002B0FD115490B608C
:102990000CE0152B04D0192B08D10021124B04E0B8
:1029A0000021124B01E0124B0021196003280FD0C7
:1029B00004D800280FD10F490A4B0BE0152804D08A
:1029C000192808D10C49084B04E00A49074B01E0DB
:1029D0000A49074B1960107010BDC046F20600206E
:1029E0003480044040A0044054D0044018C0044047
:1029F00004900440130300001304000013020000BD
:102A000038B50E4B1A680023510514D50C4C1A2802
:102A100010D80C2343430B4A0B4D9958D3181B7AFB
:102A2000216001212B70FEF725FB23682A781A729A
:102A3000012300E02360181C38BDC04634800440E8
:102A4000AC0600200C520000F30600200020704766
:102A5000F8B5214B071C1B685A053BD51F4B1B685B
:102A6000002B02D01E4A12781A711E4E00233478B1
:102A70003F220134A2425B415B421C401A4D2B783D
:102A8000A3421CD1FFF7C8FD402813DC174A137975
:102A90005BB2002BF2DA2B78002101333F20984201
:102AA000494149420B401249C95CDBB2C9B2D171FC
:102AB0002B70E3E7FF28E1DDFFF754FDDEE70C4B69
:102AC000FFB21F550B4B01221A70084BE4B2AC2227
:102AD0003470DA70F8BDC0463480044038070020F6
:102AE000340700203C0700203607002000A00640E5
:102AF000B2060020B006002038B5041C4518AC42D0
:102B000004D02078FFF7A4FF0134F8E738BDFFFFB9
:102B100008B5044B1B78002B02D0FFF723FDF8E724
:102B200008BDC046B0060020064B074A1B78107847
:102B3000DBB2C0B2834201D33F3000E00138C01A9B
:102B40007047C0463C07002036070020054B187828
:102B5000054BC0B21B78DBB2984200D24030C01A9D
:102B60007047C04635070020B106002010B5124B53
:102B700012491A780B78D2B2DBB29A4219D00133DB
:102B80003F2400209C424041404203400C48DCB2BC
:102B9000C05C0C700B49C0B2096800290BD09A4286
:102BA00000D24032D31A1A2B05DC074B1B780B726C
:102BB00001E00120404210BD35070020B106002091
:102BC000F4060020AC060020F30600200A4B1A7819
:102BD0000A4B1B78DBB29A420AD0013300223F2114
:102BE0009942524152421340054AD05CC0B201E0C2
:102BF000012040427047C04635070020B106002042
:102C0000F4060020064B1A78064BD2B21A70064B17
:102C10001B68002B02D0054A12781A727047C04612
:102C2000B106002035070020AC060020F306002086
:102C300030B5254A1379990612D52449D4790B78F1
:102C4000002001333F259D4240414042034020483F
:102C5000E4B20078834203D01E48C454DBB20B7048
:102C6000D178194CC9B24BB2002B1ADA23795BB276
:102C7000002B16DA184B19481D780378DBB29D42F9
:102C800002D16C23E3700CE0013300243F259D4208
:102C9000644164422340124CE45CDBB2E4B2D47180
:102CA0000370402319420ED0117919420BD00D4BFD
:102CB000002119700C4B1B688B4202D00B4909781C
:102CC00019722C23D37030BD00A0064035070020B8
:102CD000B1060020F40600203C0700203607002043
:102CE000B2060020B006002038070020340700207C
:102CF000164B8022196812010A431A60144A0023F5
:102D00001370144A14491370144A1370144A137040
:102D1000144A1370144A1160144AD12189001160B9
:102D2000134AC104C90EC0B21170507093702C23A5
:102D3000D370104B104A19680A408021C9010A4318
:102D40001A600E4B802292011A6070473480044052
:102D5000B00700204507002013030000B80700203B
:102D6000B1070020440700200CB0044010B004401C
:102D700000B006400CE400E0FF00FFFF00E100E0CF
:102D800010B5174B132299789143032202400A434E
:102D9000410701D510210A439A700F2210490240C1
:102DA000042A03D18A79402422438A715A79102156
:102DB0008A43084200D00A435A71997910229143FC
:102DC000840600D51143064A9971C10506D553788A
:102DD00011782020DBB201431170537010BDC04642
:102DE00000B0064008B5124B1B681A051ED5114BE2
:102DF0001B78DBB2002B02D0FFF7B4FBF7E70E4ADB
:102E00008021890111600D4A0D49D3700422FF32DF
:102E10000A600C490A600C4A13700C4A13700C4B80
:102E20001B68002B02D00B4A12781A7108BDC046ED
:102E3000348004404407002080E100E000B00640F8
:102E40000CB0044010B00440B0070020450700203B
:102E5000400700206E07002038B5041C0B4B1D787E
:102E6000EDB2002DFAD1201C0121FEF703F9291C37
:102E7000201CFEF7CDF80C225443054B054AE158BF
:102E80001C191160044B227A1A7038BD44070020C7
:102E90000C520000B4070020AF07002070477047B5
:102EA00038B50E4B1A680023110514D50C4C1A289E
:102EB00010D80C2343430B4A0B4D9958D3181B7A57
:102EC000216001212B70FEF7D5F823682A781A7249
:102ED000012300E02360181C38BDC0463480044044
:102EE000400700200C5200006E07002000207047B1
:102EF000F8B5214B071C1B681A053BD51F4B1B68F7
:102F0000002B02D01E4A12781A711E4E002334780C
:102F100027220134A2425B415B421C401A4D2B78B0
:102F2000A3421CD1FFF778FB402813DC174A137922
:102F30005BB2002BF2DA2B78002101332720984274
:102F4000494149420B401249C95CDBB2C9B2D17157
:102F50002B70E3E7FF28E1DDFFF704FBDEE70C4B16
:102F6000FFB21F550B4B01221A70084BE4B2AC2282
:102F70003470DA70F8BDC04634800440B4070020D5
:102F8000AF070020B8070020B107002000B00640BE
:102F9000460700204407002038B5041C4518AC4201
:102FA00004D02078FFF7A4FF0134F8E738BDFFFF15
:102FB00008B5044B1B78002B02D0FFF7D3FAF8E7D3
:102FC00008BDC04644070020064B074A1B7810780E
:102FD000DBB2C0B2834201D3273000E00138C01A0F
:102FE0007047C046B8070020B1070020054B18788D
:102FF000054BC0B21B78DBB2984200D24030C01AF9
:103000007047C046B00700204507002010B5124B9E
:1030100012491A780B78D2B2DBB29A4219D0013336
:103020003F2400209C424041404203400C48DCB217
:10303000C05C0C700B49C0B2096800290BD09A42E1
:1030400000D24032D31A1A2B05DC074B1B780B72C7
:1030500001E00120404210BDB007002045070020DC
:103060006F070020400700206E0700200A4B1A78E7
:103070000A4B1B78DBB29A420AD0013300223F216F
:103080009942524152421340054AD05CC0B201E01D
:10309000012040427047C046B0070020450700208D
:1030A0006F070020064B1A78064BD2B21A70064BF7
:1030B0001B68002B02D0054A12781A727047C0466E
:1030C00045070020B0070020400700206E070020C1
:1030D00030B5254A1379990612D52449D4790B784D
:1030E000002001333F259D4240414042034020489B
:1030F000E4B20078834203D01E48C454DBB20B70A4
:10310000D178194CC9B24BB2002B1ADA23795BB2D1
:10311000002B16DA184B19481D780378DBB29D4254
:1031200002D16C23E3700CE00133002427259D427B
:10313000644164422340124CE45CDBB2E4B2D471DB
:103140000370402319420ED0117919420BD00D4B58
:10315000002119700C4B1B688B4202D00B49097877
:1031600019722C23D37030BD00B00640B007002088
:10317000450700206F070020B8070020B107002096
:103180004607002044070020B4070020AF070020B6
:10319000204B8022196852010A431A601E4A0023FC
:1031A00013701E4A13701E4A13701E4A13701E4A73
:1031B00013701E4B1B78062B04D0072B05D11C4A1D
:1031C0001C4B01E01A4A1C4B1A601C4B1B78082B45
:1031D00005D0142B07D1D1229200194B02E0D12245
:1031E000184B92001A60184BC204D20E1A70C0B26B
:1031F000002258709A702C22DA70144B144A196805
:103200000A408021C9030A431A60124B8022D2016E
:103210001A607047348004402C080020C107002049
:10322000340800202D080020C007002005030020DE
:103230001303000008C0044010C00440060300202F
:1032400014C004400CC0044000C006400CE400E080
:10325000FFFF00FF00E100E010B5174B1322997843
:103260009143032202400A43410701D510210A433A
:103270009A700F2210490240042A03D18A7940240F
:1032800022438A715A7910218A43084200D00A43A6
:103290005A71997910229143840600D51143064A48
:1032A0009971C10506D5537811782020DBB201430E
:1032B0001170537010BDC04600C0064008B5124BD7
:1032C0001B68DA041ED5114B1B78DBB2002B02D031
:1032D000FFF748F9F7E70E4A8021C90111600D4A4E
:1032E0000D49D3700422FF320A600C490A600C4A6F
:1032F00013700C4A13700C4B1B68002B02D00B4A46
:1033000012781A7108BDC04634800440C0070020FE
:1033100080E100E000C0064008C004400CC004404A
:103320002C080020C1070020BC070020EA0700206D
:1033300038B5041C0B4B1D78EDB2002DFAD1201CC2
:103340000121FDF797FE291C201CFDF761FE0C22D0
:103350005443054B054AE1581C191160044B227A6D
:103360001A7038BDC00700200C5200003008002041
:103370002B08002030B5002901D080231843154ABE
:103380001378141C984224D0134A1268D5041FD510
:103390007F221340082B04D0142B05D100220F4BA1
:1033A00001E00F4B00221A604423002900D0602363
:1033B0007F220240082A06D0142A09D1C022920096
:1033C0001343064A03E0C02292001343044A1360E9
:1033D000207030BD060300203480044014C0044037
:1033E0000CC0044010B50F4A1378984218D00E490B
:1033F0000968CC0413D5062B04D0072B05D1002176
:103400000A4B01E00A4B00211960062804D0072866
:1034100005D10849054B01E00649054B19601070BC
:1034200010BDC046050300203480044008C004409D
:1034300010C004401303000038B50E4B1A68002377
:10344000D10414D50C4C1A2810D80C2343430B4A32
:103450000B4D9958D3181B7A216001212B70FDF771
:1034600009FE23682A781A72012300E02360181CE1
:1034700038BDC04634800440BC0700200C52000018
:10348000EA07002000207047F8B5214B071C1B6895
:10349000DA043BD51F4B1B68002B02D01E4A127862
:1034A0001A711E4E0023347827220134A2425B4158
:1034B0005B421C401A4D2B78A3421CD1FFF7ACF89D
:1034C000402813DC174A13795BB2002BF2DA2B7811
:1034D0000021013327209842494149420B401249BB
:1034E000C95CDBB2C9B2D1712B70E3E7FF28E1DD23
:1034F000FFF738F8DEE70C4BFFB21F550B4B0122EC
:103500001A70084BE4B2AC223470DA70F8BDC046D1
:1035100034800440300800202B08002034080020AC
:103520002D08002000C00640C2070020C007002070
:1035300038B5041C4518AC4204D02078FFF7A4FF2E
:103540000134F8E738BDFFFF08B5044B1B78002BAA
:1035500002D0FFF707F8F8E708BDC046C007002013
:10356000064B074A1B781078DBB2C0B2834201D306
:10357000273000E00138C01A7047C04634080020E8
:103580002D080020054B1878054BC0B21B78DBB224
:10359000984200D24030C01A7047C0462C08002024
:1035A000C107002010B5124B12491A780B78D2B21D
:1035B000DBB29A4219D001333F2400209C424041A3
:1035C000404203400C48DCB2C05C0C700B49C0B2F6
:1035D000096800290BD09A4200D24032D31A1A2B24
:1035E00005DC074B1B780B7201E00120404210BD47
:1035F0002C080020C1070020EB070020BC0700209A
:10360000EA0700200A4B1A780A4B1B78DBB29A4271
:103610000AD0013300223F219942524152421340C5
:10362000054AD05CC0B201E0012040427047C0466C
:103630002C080020C1070020EB070020064B1A7859
:10364000064BD2B21A70064B1B68002B02D0054AFB
:1036500012781A727047C046C10700202C0800205B
:10366000BC070020EA07002030B52E4A13799906DE
:1036700024D52D49D4790B78002001333F259D4274
:103680004041404203402948E4B20078834203D0DD
:103690002748C454D8B208702649086800280DD0BD
:1036A00025490978C9B28B4201D35B1A01E05B1A44
:1036B0004033272B02DD214B1B780371D178194C45
:1036C000C9B24BB2002B1ADA23795BB2002B16DA9F
:1036D0001B4B19481D780378DBB29D4202D16C2345
:1036E000E3700CE00133002427259D4264416442CD
:1036F0002340144CE45CDBB2E4B2D4710370402389
:1037000019420ED0117919420BD00F4B00211970BC
:103710000E4B1B688B4202D00D49097819722C237D
:10372000D37030BD00C006402C080020C107002027
:10373000EB070020BC0700202D080020EA0700202E
:1037400034080020C2070020C007002030080020F5
:103750002B0800201FB572B6154B70221A70154A3F
:1037600041211170144A0F21117080221A701A78A9
:1037700052B2002AFBDA114B186862B6104B98421D
:1037800001D80A23584301AC211C0A22FEF770FF1E
:103790000023E15C0B4A002905D0580010180133C2
:1037A00041800A2BF5D101335B0013701FBDC04669
:1037B00000000240070002400600024008000240EC
:1037C0007F969800E403002008B50368C9B21B681F
:1037D000984708BD08B50368C9B21B68984708BD7B
:1037E00008B50368C9B21B68984708BD08B50368E7
:1037F000C9B21B68984708BD08B5044B4808C018F3
:1038000000F0A2FAFEF75CFF08BDC046C0C62D005E
:1038100010B5064B4808C018141C00F095FAFEF7C6
:103820004FFF201CFEF7C0FF10BDC046C0C62D00D4
:1038300008B5FEF7EBFF08BD08B5081CFFF720F838
:1038400008BD08B5081CFFF793F808BD08B5081CAB
:10385000111CFFF737F808BD08B5081CFFF7D0F8B2
:10386000431E9841C0B208BD08B5081CFFF7EEF82A
:10387000431E9841C0B208BD08B5FFF767F908BDFF
:1038800008B5FFF7A3F908BD08B5FFF76FF908BD44
:1038900008B5FFF73DF908BD08B5FFF7B3F908BD56
:1038A00008B5FFF741F908BD08B5081CFFF7D0F8C7
:1038B000012008BD08B5081CFFF7CAF8012008BDA3
:1038C00010B5081C141C111CFFF716F9201C10BDA4
:1038D00038B5081C0D1C01F041F9041C211C281CE2
:1038E000FFF70AF9201C38BD7047FFFF044B002288
:1038F0001A711A73FA21034A890099601A60704795
:1039000038080020E053000008B50368C9B21B68FE
:10391000984708BD08B50368C9B21B68984708BD39
:1039200008B50368C9B21B68984708BD08B50368A5
:10393000C9B21B68984708BD08B5044B4808C018B1
:1039400000F002FAFFF7D4F908BDC04660E31600A4
:1039500010B5064B4808C018141C00F0F5F9FFF725
:10396000C7F9201CFFF70CFA10BDC04660E3160033
:1039700008B5FFF737FA08BD08B5081CFFF76CFA61
:1039800008BD08B5081CFFF78AFA08BD08B5081C71
:10399000111CFFF783FA08BD08B5081CFFF780FA71
:1039A000431E9841C0B208BD08B5081CFFF79EFA37
:1039B000431E9841C0B208BD08B5FFF717FB08BD0C
:1039C00008B5FFF753FB08BD08B5FFF71FFB08BD9F
:1039D00008B5FFF7EDFA08BD08B5FFF763FB08BDB2
:1039E00008B5FFF7F1FA08BD08B5081CFFF780FA23
:1039F000012008BD08B5081CFFF77AFA012008BDB0
:103A000010B5081C141C111CFFF7C6FA201C10BDB1
:103A100038B5081C0D1C01F0A1F8041C211C281C41
:103A2000FFF7BAFA201C38BD7047FFFF044B002295
:103A30001A711A73FA21034A890099601A60704753
:103A4000480800204054000008B50368C9B21B684C
:103A5000984708BD08B50368C9B21B68984708BDF8
:103A600008B50368C9B21B68984708BD08B5036864
:103A7000C9B21B68984708BD08B5044B4808C01870
:103A800000F062F9FFF784FB08BDC04660E3160052
:103A900010B5064B4808C018141C00F055F9FFF784
:103AA00077FB201CFFF7D8FB10BDC04660E3160073
:103AB00008B5FFF703FC08BD08B5081CFFF738FC84
:103AC00008BD08B5081CFFF78DFC08BD08B5081C2B
:103AD000111CFFF74FFC08BD08B5081CFFF7ACFC34
:103AE000431E9841C0B208BD08B5081CFFF7CAFCC8
:103AF000431E9841C0B208BD08B5FFF743FD08BD9D
:103B000008B5FFF77FFD08BD08B5FFF74BFD08BD01
:103B100008B5FFF719FD08BD08B5FFF78FFD08BD13
:103B200008B5FFF71DFD08BD08B5081CFFF7ACFC84
:103B3000012008BD08B5081CFFF7A6FC012008BD40
:103B400010B5081C141C111CFFF7F2FC201C10BD42
:103B500038B5081C0D1C01F001F8041C211C281CA0
:103B6000FFF7E6FC201C38BD7047FFFF044B002226
:103B70001A711A73FA21034A890099601A60704712
:103B800058080020A054000008B50B4B1A68002A02
:103B900004D001221A60094B1B689847084B1B7818
:103BA000002B08D0074B1A68002A04D001221A60A3
:103BB000024B5B68984708BD0C7103406C080020FD
:103BC0006A0800201C710340064B80221968120409
:103BD0000A431A60044B00221A60044B01221A7037
:103BE0007047C0463C800440007003406A080020D3
:103BF000054B01221A60054B054A19680A401A60F4
:103C0000044B00221A707047007003403C8004404F
:103C1000FFFF7FFF6A08002070B544780E4D0F4EFD
:103C200023015A199B190E4D0669A4004260665182
:103C3000002483601C60116003221A60094B417BE1
:103C4000094A1868090402400A431A60074B802297
:103C5000D2031A6070BDC046007103400871034072
:103C60006C08002014E400E0FFFF00FF00E100E02A
:103C7000F8B50C4B061C1B780F1C002B01D1FFF76D
:103C8000A3FF094D2C78002C04D06B7800208342D0
:103C900007D10124301C7470391CFFF7BDFF0120CF
:103CA0002855F8BD6A0800206808002008B5836818
:103CB00000221A608021074BC90319604178064B26
:103CC0005A541A78002A04D15B78002B01D1FFF7EF
:103CD0008FFF08BD80E100E06808002070B5037820
:103CE000041C0E1C151C002B03D0FFF7DFFF002364
:103CF00023702661201C291CFFF7BAFF002802D080
:103D00000123237000E02070207870BD037810B587
:103D1000041C002B01D0FFF7C9FF0023237010BD46
:103D200002B4714649084900095C49008E4402BC4E
:103D30007047C04603B47146490840004900095A1B
:103D400049008E4403BC7047002934D0012300226F
:103D500010B488422CD301242407A14204D281420A
:103D600002D209011B01F8E7E400A14204D281421A
:103D700002D249005B00F8E7884201D3401A1A4397
:103D80004C08A04202D3001B5C0822438C08A042CE
:103D900002D3001B9C082243CC08A04202D3001B84
:103DA000DC082243002803D01B0901D00909E3E7FE
:103DB000101C10BC7047002801D00020C04307B47D
:103DC000024802A14018029003BDC046190000003D
:103DD0000029F0D003B5FFF7B9FF0EBC4243891AA2
:103DE0001847C0467047C0468446081C6146FFE736
:103DF0001FB500F001FA002801D40021C8421FBD00
:103E000010B500F087F94042013010BD10B500F048
:103E1000F3F9002801DB002010BD012010BDC046D1
:103E200010B500F0E9F9002801DD002010BD0120E7
:103E300010BDC04610B500F097F9002801DC002045
:103E400010BD012010BDC04610B500F08DF900284E
:103E500001DA002010BD012010BDC0461C21012345
:103E60001B04984201D3000C10391B0A984201D35D
:103E7000000A08391B09984201D30009043902A23B
:103E8000105C40187047C0460403020201010101A2
:103E900000000000000000009E2110B5C905041CB0
:103EA000FFF7D2FF002803D1201C00F091FC10BDC9
:103EB0009E21C905201C00F015FB00F089FC802321
:103EC0001B06C018F3E7C046F0B55F4656464D46A0
:103ED0004446F0B446024500C00F85B00F1C760A78
:103EE0002D0E804641D0FF2D26D0802424040021B1
:103EF0002643F6007F3D89468B46F90F7C02780009
:103F0000640A000E00918A463CD0FF2834D08023FA
:103F10001B041C430023E4007F380193009F4346A9
:103F2000019A7B4049469C4611430F2900D971E014
:103F3000764F89007F58BF46002E3ED108220223CB
:103F400091469B46D9E75A46341CC24601920199D4
:103F5000022937D0032900D1CFE0012900D0ABE0FE
:103F600053460B400022002632E0002E19D10421D6
:103F7000012289469346C0E7221C531E9A41023211
:103F80000192CBE701270197002CC7D0201CFFF737
:103F900065FF431F9C4076235B420021181A019164
:103FA000BCE7301CFFF75AFF7625431F9E406D4249
:103FB00000232D1A99469B469FE70C23032199461F
:103FC0008B469AE7D446012367463B40FF220026F2
:103FD0007602D205700ADB071043184305B03CBCDB
:103FE00090469946A246AB46F0BD80260023F603D4
:103FF000FF22EDE700220026EAE78020C003064208
:104000003BD0044239D1061C26437602760A009B37
:10401000FF22DDE7281A039076016401A64239D316
:10402000361B1A2201230120311C5B007600002977
:1040300001DBB44201D8361B0343013A002AF3DC0A
:10404000741EA641341C1C43039A7F32002A27DDCC
:10405000630704D00F232340042B00D0043427012E
:1040600003D52B4B039A1C408032FE2A0BDD012323
:1040700061460B40FF220026AAE706437602760A35
:104080004346FF22A4E7A40101236746660AD2B291
:104090003B409DE7039F1B22013F03970023C2E79C
:1040A0007E23039F5B42DB1B1B2B07DD0123614645
:1040B0000B40002200268BE7D446C5E7221CDA40DD
:1040C000039B9E339C40231C5C1EA34113435A0751
:1040D00004D00F221A40042A00D004335F0105D512
:1040E000012361460B400122002671E79E016246D2
:1040F00001231340760A00226AE78026F60326434E
:104100007602760A5346FF2262E7C046F854000062
:10411000FFFFFFF74A02430270B55C0A550A4300ED
:104120004A001B0EC60F120EC90FFF2B05D0FF2A27
:1041300008D0012093420BD070BD0120002CFBD190
:10414000FF2AF6D10120002DF6D101209342F3D1B0
:10415000AC42F1D18E4205D0002BEDD1201C441E83
:10416000A041E9E70020E7E74A024302F0B55C0A14
:10417000550A43004A001B0EC60F120EC90FFF2B33
:1041800031D0FF2A34D0002B16D1604260418446E2
:10419000002A14D0002820D18E4217D1934215DC7A
:1041A00004DBAC4212D80020AC4212D27042704103
:1041B0004042012318430CE0002AEDD194466F429F
:1041C0006F416046002805D1002FE5D070420123E1
:1041D0001843F0BD0020002FFBD148424841404227
:1041E00001231843F5E7002CCBD002204042F0E732
:1041F000002DC8D0F9E7C0464A024302F0B55C0A78
:10420000550A43004A001B0EC60F120EC90FFF2BA2
:1042100027D0FF2A29D0002B10D0002A15D1944690
:104220006F426F416046002815D00020002F04D156
:1042300048424841404201231843F0BD604260417A
:104240008446002AECD00028F2D18E4211D0704270
:1042500001231843F1E7002FF7D0704201231843E0
:10426000EBE70220002CE8D1D3E70220002DE4D1B7
:10427000D1E79342EBDC04DBAC42E8D80020AC424F
:10428000DBD270427041404201231843D5E7C0465B
:10429000F0B55F4656464D464446F0B444024600EB
:1042A00083B00F1C640A360EC50F002E41D0FF2EBE
:1042B00022D080231B0400201C43E4007F3E824662
:1042C0008046391C4B007F02C90F7F0A1B0E8B46AC
:1042D0003BD0FF2B34D0802212041743FF007F3BDA
:1042E00000215A466A40019252460A430F2A63D877
:1042F0007A48920082589746002C3FD10822022328
:1043000092469846DDE70195404602282AD1019A57
:1043100001251540FF2300246402DB05600AED0738
:104320001843284303B03CBC90469946A246AB468E
:10433000F0BD002C27D10420012282469046C0E720
:10434000391C4A1E91410231CBE70121002FC8D010
:10435000381CFFF783FD431F9F4076235B421B1AE7
:104360000021BEE7032800D1AEE001284FD101981B
:1043700042461040C5B200230024CDE70C230320A1
:104380009A4680469DE7201CFFF768FD7626431F6E
:104390009C4076420023361A9A46984691E780243C
:1043A0000025E403FF23B7E75B463C1C01938846E6
:1043B000AAE73C1C8846A7E7250C24043A0C240CE9
:1043C0003F04F6183F0C211C231C794353436F43D1
:1043D0005543FB180A0C9B18B1469F4202D9802214
:1043E0005202AD1809041A04090C521894011B0C4E
:1043F000611E8C41920EED181443AD012C43230134
:1044000005D5012263080120144081441C434B461A
:104410007F33002B2DDD600704D00F222240042AB9
:1044200000D00434220103D52D4B1C404B46803371
:10443000FE2B17DD019B01251D400024FF236BE7A8
:104440008020C003044208D0074206D1041C3C432C
:104450006402640A5D46FF235EE704436402640A63
:10446000FF2359E70198A4010125640ADBB2054046
:1044700052E77E235B424A469B1A1B2B05DD019BBC
:1044800001251D400024002346E7221CDA404B464C
:104490009E339C40231C5C1EA3411343580704D049
:1044A0000F221A40042A00D004335A0105D5019B7B
:1044B00001251D40002401232EE701989C010125C0
:1044C000640A0540002327E78027FF03019B3C4344
:1044D000640201251D40640AFF231DE738550000D2
:1044E000FFFFFFF7F8B5C20F430244004D0248003A
:1044F000240E161C9B09000EC90FAD09FF2800D120
:1045000083E0012779408A425CD0221A002A00DC2D
:104510008EE000281ED1002D00D07AE0580704D08C
:104520000F221A40042A00D004338021C90401223A
:104530001940324000293AD00134FF2C00D183E0E9
:104540009B015B0A5B02E4B2E405580AD2072043F0
:104550001043F8BDFF2CE1D08021C9040D431B2A74
:1045600000DD31E1291C2020D140821A95406A1ECD
:1045700095410D435B1B5801D0D59B019F09381C09
:10458000FFF76CFC421F974094425FDC141B1F2313
:104590001B1B3A1C9F40611C3B1CCA405F1EBB4159
:1045A00013430024BAE7131EB8D100230022DB080E
:1045B000FF2C04D1002B47D08020C00303435B02B3
:1045C0005B0ABFE7211A002944DD002827D0FF2C11
:1045D000A4D08020C00405431B2900DDF2E0281C84
:1045E0002027C840791A8D40691E8D4105435B190B
:1045F000590100D492E70134FF2C59D073490122AC
:104600001A400B405B08134388E7002D00D07AE77F
:1046100077E7013A002AADD0FF2CA0D17EE7002D2C
:1046200000D17BE701390029E1D0FF2CD4D175E717
:10463000002A1BD1621CD2B2012A4BDD5F1B7A011A
:1046400023D5EF1A0E1C9AE700237BE75F4BA41AD1
:104650003B4063E7002946D1611CC8B2012829DD2F
:10466000FF2924D0EB185B080C1C57E7002C13D053
:10467000FF2818D08024E404524223431B2A4DDD36
:104680000123EB1A041C0E1C75E7002F00D076E7FF
:104690000023002200248AE7002B3BD0D243002ACB
:1046A000EFD0FF28EAD12B1CFF240E1C36E7FF2495
:1046B00000237CE7002C5CD1002B00D180E0002D92
:1046C00000D12BE75B19580100D427E73F4A0124AA
:1046D000134023E7002C15D1002B40D1002D63D0CF
:1046E0002B1C0E1C1AE7002C21D1002B54D0C943DF
:1046F000002904D0FF284CD01B2958DD01235B1969
:10470000041C75E7002B19D1002D48D02B1C0E1C62
:10471000FF2403E72B1C041C0E1CFFE61C1C202698
:10472000D440B21A93405A1E93412343A9E7FF286D
:104730002FD08024E40449422343DDE7FF24002DE9
:1047400000D1EBE68022DB08D203134204D0ED084F
:10475000154201D12B1C0E1CDB00FF24DEE6002DD0
:1047600000D1DBE65A1B500100D41CE7EB1A0E1CEB
:10477000D4E6002B0DD0FF24002D00D1CEE6802200
:10478000DB08D2031342E7D0ED081542E4D12B1C1D
:10479000E2E72B1CFF24C1E62B1C041CBEE6802391
:1047A00000229B04FF2402E7231C0022FFE61C1CBE
:1047B0002027CC40791A8B40591E8B4123439EE71A
:1047C0002B1CABE6012512E70125D3E6FFFFFFFB1B
:1047D0004302590A4300C20F1B0E00207E2B0DDD41
:1047E0009D2B0CDC802000040143952B0ADC9620D5
:1047F000C31AD9404842002A00D1081C7047034B15
:10480000D018FBE7963B9940F4E7C046FFFFFF7FD7
:1048100010B5041E33D0FFF721FB9E231B1A962BE5
:1048200009DC083884406402640ADBB26402DB05F8
:10483000600A184310BD992B0ADD0522121A211CAB
:10484000D1400A1C011C1B318C40611E8C41144359
:10485000052801DD421F9440144A2240610704D01C
:104860000F210C40042C00D0043251010AD59F23A3
:10487000181AFF2816D09401640AC3B2D6E70023A1
:104880000024D3E7D208FF2B03D05402640ADBB222
:10489000CCE7002A06D08024E40314436402640AAF
:1048A000FF23C3E7FF230024C0E7C046FFFFFFFB51
:1048B00008B5031C081C191C00F002F808BDFFFF16
:1048C00038B5051C05480C1C131C002804D0022018
:1048D000291C221C00E000BF38BDC04600000000BB
:1048E00070B50E4B0E4D0024ED1AAD101E1CAC42DF
:1048F00004D0A300F35898470134F8E700F058FEBD
:10490000084B094D0024ED1AAD101E1CAC4204D01A
:10491000A300F35898470134F8E770BDBC55000078
:10492000BC550000BC550000D855000008B5034B2D
:10493000011C186800F02EF808BDC0465C04002079
:1049400010B50023934203D0CC5CC4540133F9E783
:1049500010BD70B5814201D300230CE08C18A04239
:10496000FAD28518131C013B0BD351426618F65C32
:104970006918CE54F7E7934203D0CC5CC45401339A
:10498000F9E770BD031C8218934202D019700133FD
:10499000FAE7704730B5002940D004390B68002B86
:1049A00000DAC9181E4A1368141C002B02D14B6090
:1049B000116033E099420FD208680A189A4205D173
:1049C00013685268C01808604A6000E04B602160BC
:1049D00024E08A4203D8131C5A68002AF9D11D68C2
:1049E0005C198C420BD109686918581819609042FB
:1049F00014D114685268091919605A600EE08C428B
:104A000002D90C23036009E008680C18944203D112
:104A100014685268001908604A60596030BDC04689
:104A20007808002070B50323CD1C9D430835061C73
:104A30000C2D01D20C2501E0002D3FDB8D423DD332
:104A4000204B1C681A1C211C002913D00868431B2A
:104A50000DD40B2B02D90B60CC181EE08C4202D176
:104A6000636813601AE0486860600C1C16E00C1C58
:104A70004968E9E7144C2068002803D1301C00F095
:104A800031F82060301C291C00F02CF8431C15D094
:104A9000C41C03239C4384420AD12560201C0B3094
:104AA0000722231D9043C31A0BD05A42E25008E05C
:104AB000211A301C00F016F80130EED10C233360BF
:104AC000002070BD780800207408002008B50A1C7A
:104AD0000349031C0868191C00F02DFB08BDC046E3
:104AE0005C04002038B5074C0023051C081C23601B
:104AF000FDF78AFD431C03D12368002B00D02B60F7
:104B000038BDC046D40800200EB400B59CB01DAB23
:104B100004CB822202A992008A810A4A02908A600A
:104B20004A6101225242CA81074A086110681D9AEF
:104B3000019300F07BF8029A002313701CB008BCAC
:104B400003B01847FFFFFF7F5C040020031C0A78B6
:104B500001311A700133002AF9D170470023C25C79
:104B60000133002AFBD1581E7047FFFFF0B58D6856
:104B700085B0071C0C1C03920193AB4245D39022D5
:104B80008B89D20013423DD06269032656430969DE
:104B90002068F20F401A96190290021C0198013207
:104BA00012187610964200D2161C381C5A050FD5E2
:104BB000311CFFF737FF051E13D0029A2169FFF75A
:104BC000BFFEA289184B134080221343A38111E03A
:104BD000321C00F0B0FA051E0CD1381C2169FFF719
:104BE000D9FE0C233B60A389402213430120A381FB
:104BF000404217E0029B2561ED1825606661019D2A
:104C0000F61AA6600198A84200D2019D2A1C2068CD
:104C10000399FFF79EFEA2680020531BA360236840
:104C20005D19256005B0F0BD7FFBFFFFF0B59FB0BB
:104C3000039005938B890E1C171C19060FD532693A
:104C4000002A0CD14021FFF7EDFE306030610028D2
:104C500003D103990C230B60C9E04023736106ADB7
:104C600000236B6120236B763023AB763C1C2378CA
:104C7000002B03D1E21B029211D003E0252BF9D0C7
:104C80000134F4E70398311C3A1C029BFFF76EFFD6
:104C9000013000D1A6E06969029A8B186B61237814
:104CA000002B00D19EE0012252426A606A46002336
:104CB0005B3201342B60EB60AB601370AB654E4F21
:104CC0002178381C052200F02BFA002807D0C71BDA
:104CD0002B680120B840184328600134EFE72B68A7
:104CE000D90603D56A4620215B3211701A0703D515
:104CF0006A462B215B32117022782A2A01D0099B47
:104D00000EE0059A111D12680591002A01DB099237
:104D100004E05242EA60022213432B60013409E0AE
:104D20002278303A092A04D80A214B4301349B18CF
:104D3000F6E7099323782E2B18D163782A2B09D113
:104D4000059B02341A1D1B680592002B0DDA012306
:104D50005B420AE0013400232278303A092A04D861
:104D60000A214B4301349B18F6E70793234F217820
:104D7000381C032200F0D4F9002806D0C71B2B688A
:104D80004020B84018432860013421781C4806228E
:104D9000671C297600F0C4F9002812D0194B002BAB
:104DA00006D1059B0722073393430833059314E08C
:104DB00005AB00930398291C321C134B00E000BF85
:104DC00007E005AB00930398291C321C0E4B00F042
:104DD00091F804900499013104D06A690499531838
:104DE0006B6143E7B3895A0601D40B9801E00120B7
:104DF00040421FB0F0BDC0467A550000805500000B
:104E000084550000000000006D4B0000F7B5151C34
:104E100001930A698B68061C0C1C934200DA131C70
:104E2000221C2B6043321278002A01D001332B6000
:104E30002068800602D52B6802332B602168062784
:104E40000F401FD0231C43331B785A1E9341226806
:104E500092061FD5E11840313020C870211C5A1C21
:104E600045310978A21840320233D17012E0221C79
:104E7000301C019919320123089FB847013011D025
:104E8000009F01370097E0682968009F431A9F42FE
:104E9000EDDBD7E7221C301C01994332089FB8474D
:104EA000013002D10120404223E0206806212B6816
:104EB000E26801400025042903D1D51AEB43DB1732
:104EC0001D40A26823699A4201DDD31AED1800271C
:104ED0000097009FAF420BDA221C301C01991A3256
:104EE0000123089FB8470130DCD0009F0137EFE76E
:104EF0000020FEBDF0B50D1C8BB043350692059029
:104F0000079304950B7E0C1C109A6E2B00D1A7E022
:104F100011D8632B22D009D8002B00D1B0E0582B38
:104F200000D0C0E045310B707B4D4EE0642B1CD0AF
:104F3000692B1AD0B7E0732B00D1A5E009D86F2BED
:104F400029D0702B00D0AEE00E68202333430B60D5
:104F500036E0752B1FD0782B32D0A4E013680D1CDF
:104F6000191D423511601B689FE0216813680E0609
:104F700003D5191D11601E6805E04806F9D5191DF5
:104F8000116000215E5E644B002E3BDA049D2D22F1
:104F900076422A7036E0216813680E0603D5191D83
:104FA00011601E6804E04806F9D5191D1E881160BD
:104FB000594B227E039308276F2A1ED00A271CE034
:104FC000231C78214533554D197011682368081D3D
:104FD000039510601E0601D50E6802E05806FBD549
:104FE0000E88D90702D52022134323601027002EF4
:104FF00003D1226820239A432260231C00224333DA
:105000001A7001E003930A276368A360002B03DB97
:105010002568042295432560002E02D1049D002BB3
:105020000ED0049D301C391CFEF7D2FE0398013DC2
:10503000435C301C2B70391CFEF786FE061EF1D136
:10504000082F09D12168C90706D5626823699A42E9
:1050500002DC013D30232B70049E731B23612AE088
:10506000086813684969050604D5181D10601B6897
:10507000196005E04606F8D5181D10601B681980F8
:1050800000232361049D16E01368191D11601D683B
:10509000281CFFF763FD63682061984200D92361F3
:1050A0002069606004E0251C42352B7001232361D8
:1050B000049E00233370079E05980096211C09AAC0
:1050C000069BFFF7A3FE013002D10120404221E000
:1050D0002A1C059806992369079DA8470130F4D03A
:1050E0002668B60705D4099BE068984212DA181CB6
:1050F00010E00025E0680999431A9D42F3DA221C6A
:105100000598069919320123079EB0470130DCD07B
:105110000135EFE70BB0F0BD8B5500009C5500004A
:10512000C9B28218904204D003788B4202D0013079
:10513000F8E700207047F8B5061C0C1C151C002968
:1051400004D1111CFFF76EFC041C18E0002A03D1E7
:10515000FFF720FC2C1C12E000F013F8A8420ED23E
:10516000301C291CFFF75EFC071E07D0211C2A1CDF
:10517000FFF7E6FB301C211CFFF70CFC3C1C201C3D
:10518000F8BD04390B68181F002B02DAC8581B1829
:10519000181F7047256C6400256C75004720256337
:1051A00020256C6420256420256400656E640074ED
:1051B0002000360020473A002050445F7363726538
:1051C000656E3A002050445F6C617365723A005519
:1051D0006E6B6E6F776E20636F6D6D616E643A20DB
:1051E00000050E08090D0C06070F0B004417FF05FC
:1051F0000E08090D0C06070F0B004417FFFFFFFFF9
:10520000FFFFFFFFFFFFFF1A1BFFFFFF420000F839
:1052100040A0044001000000420000F844A0044007
:1052200002000000C00000F800C0044001000000BF
:10523000000000F80490044002000000000000F8A4
:105240000890044004000000C00000F81CC00440A6
:1052500080000000C00000F810C0044010000000F2
:10526000C00000F808C0044004000000C00000F8BE
:105270000CC0044008000000800000F80CB004409E
:1052800008000000800000F810B00440100000008A
:10529000800000F818B0044040000000800000F8D2
:1052A0001CB0044080000000800000F814B00440EE
:1052B00020000000C00000F804C00440020000000C
:1052C000800000F800B0044001000000400000F839
:1052D00000A0044001000000400000F804A00440C9
:1052E00002000000400000F80CA00440080000008C
:1052F000400000F808A0044004000000C00000F8CE
:1053000014C0044020000000C00000F818C0044091
:1053100040000000800000F804B0044002000000DB
:10532000800000F808B0044004000000020100F80A
:1053300050D0044010000000020100F854D0044096
:1053400020000000030100F878D004404000000075
:105350000000000000000000312500003B25000097
:105360000925000011250000192500002125000055
:1053700029250000000000001519151519FFFFFF71
:1053800000010000070300201200000000020000DE
:10539000320300209500000000030000E00300201D
:1053A00000000000010309041A03002000000000AF
:1053B00002030904C80300200000000003030904DD
:1053C000E4030020000000000000000000000000D6
:1053D00000000000FFFFFFFF0000000000000000D1
:1053E000A9380000C1380000793800008938000071
:1053F0008138000091380000F937000011380000B2
:105400003138000039380000433800004D380000C2
:10541000593800006938000099380000A1380000B0
:10542000C9370000D5370000E1370000ED37000034
:10543000D1380000B5380000000000000000000076
:10544000E9390000013A0000B9390000C93900000B
:10545000C1390000D139000039390000513900004C
:105460007139000079390000833900008D3900005E
:1054700099390000A9390000D9390000E13900004C
:105480000939000015390000213900002D390000CC
:10549000113A0000F5390000000000000000000093
:1054A000293B0000413B0000F93A0000093B0000A5
:1054B000013B0000113B0000793A0000913A0000E6
:1054C000B13A0000B93A0000C33A0000CD3A0000FA
:1054D000D93A0000E93A0000193B0000213B0000E6
:1054E000493A0000553A0000613A00006D3A000068
:1054F000513B0000353B000014400000C63F000057
:10550000F43F00004E3F0000F43F0000EA3F00007F
:10551000F43F00004E3F0000C63F0000C63F0000C1
:10552000EA3F00004E3F0000463F0000463F0000BB
:10553000463F0000FA3F0000B8430000B2430000BD
:10554000B2430000A84300000843000008430000E5
:105550009E430000A8430000084300009E43000053
:1055600008430000A8430000064300000643000073
:1055700006430000404400004300232D302B200050
:10558000686C4C00656667454647003031323334FD
:10559000353637383941424344454600303132339D
:1055A00034353637383961626364656600FFFFFF62
:1055B000F8B5C046F8BC08BC9E46704739040000E8
:1055C000B90C00002923000049250000ED38000037
:0855D0002D3A00006D3B0000C4
:1055D800000000009C04002014050020AC040020FA
:1055E8007C040020FC0400200A040000C90E00000E
:1055F800C90E0000C90E0000C90E0000C90E000047
:10560800C90E0000C90E0000C90E0000C90E000036
:10561800C90E0000C90E0000C90E0000C90E000026
:10562800C90E0000C90E0000C90E0000C90E000016
:10563800C90E0000C90E0000C90E0000C90E000006
:10564800C90E0000C90E0000C90E0000C90E0000F6
:10565800C90E0000C90E0000FFFFFFFFFF00000099
:10566800D80800200107081201010100000040C00D
:1056780016890400020102030100180354006500A2
:1056880065006E00730079006400750069006E00A3
:105698006F0009029500030100C032080B000202E6
:1056A800020104090400000102020100052400109F
:1056B800010524010101042402060524060001074E
:1056C80005810310004009040100020A00000007D8
:1056D8000502024000000705830240000009040299
:1056E8000002010300000724010001410006240212
:1056F8000101000624020202000924030103010239
:105708000100092403020401010100090505024002
:105718000000000005250101010905840240000080
:105728000000052501010300180354006500650009
:105738006E007300790020004D00490044004900C4
:10574800040309040C03000000000000000000002E
:105758000000000000000000000000000000000041
:105768000000000000000000000000000000000031
:105778000000000000000000000000007855000054
:105788000000000000000000000000000000000011
:105798000000000000000000000000000000000001
:1057A80000000000000000000000000000000000F1
:1057B800000000000000000000000000FC030020C2
:00000001FF
